:020000040000FA
:0400000071303A28F9
:08000800A000030EA100831209
:1000100081018B100B11210E8300A00E200E090010
:0C007400203084008001840A80300402E7
:10008000031C3C281230B000532183160C30850528
:1000900087018312850187010730990000309A009B
:1000A000103083168E008312603083168F00831207
:1000B0000030831691009F008312C83083168100A0
:1000C000831231309000003083168C008312103080
:1000D0008B00831600309B001C141A088312BC008E
:1000E000831610309B001C141A088312BD0083165F
:1000F0002F309B001C141A088312C3006C21831636
:1001000020309B001C141A088312C2000130C20860
:100110000319C20081018E018F010B118B100B108E
:100120008C018B17A6203119A8203521B30BA428E8
:10013000031085190314B90DF03039020319752124
:100140000F303902031971217921922864000800C7
:10015000080031110130B7008B13203037078316A8
:100160009B001C141A088312A40010303707831652
:100170009B001C141A088312A30000303707831653
:100180009B001C141A088312A2008B17321CCE2865
:1001900022090339A200A309A409A50901303702E5
:1001A000031DD7283D18D7283D143E146621013081
:1001B0003702031DE0283D1CE0283D103E146A2153
:1001C000E128B70A0230370203180800AC280130D2
:1001D000B600B300B400B500B70085018701B113C4
:1001E000A620B30B0D29031085190314B90DF030A7
:1001F000390203192B29B41F8501B41F8701B40BE1
:100200000D293708B6080319B60003190B29FF306A
:1002100085008700B6039630B400311DF0283111F7
:10022000321C17292D090339AD00AE09AF098B1314
:1002300020303707BB002F08BA003E2110303707A7
:10024000BB002E08BA003E2100303707BB002D0846
:10025000BA003E218B1785018701B70AB60102302B
:100260003702031CF0286C2108003E1C08003E10D9
:100270001030BB003D08BA003E2108008B133A083D
:1002800083161C159A0083123B0883169B00553079
:100290009D00AA309D009C1464009C184C291C11E0
:1002A00083128B170800FF30D4000230D5000C30C9
:1002B000D600BA30D7003730D800DA30D9006F30E6
:1002C000DA00B830DB000230C10008000130BD00A8
:1002D000DD140800DD100800BD013D143D18DD14DB
:1002E00008003D143E14662108003D103E146A21AA
:1002F00008005C180516DC1885165C190514DC1955
:1003000085145C1A8714DC1A07155C1B0714DC1BA8
:1003100087165D180716DD1887155C1C0512DC1C96
:1003200085125C1D0510DC1D85105C1E8710DC1E0F
:1003300007115C1F0710DC1F87125D1C0712DD1CF4
:1003400087118F08031908008F01C10B08004208AC
:10035000C1005408DE00F222D4005508DE00F2226B
:10036000D5005608DE00541CF222D6005708DE00E5
:10037000D41CF222D7005808DE00541DF222D80007
:100380005908DE00D41DF222D9005A08DE00541E9E
:10039000F222DA005B08DE00D41EF222DB005C08E9
:1003A000C6005D08C700CA0BEB295408CA008B13AE
:1003B000831640309B001C141A0883125405031D39
:1003C0005C14831650309B001C141A0883125405C9
:1003D000031D5C108B17CB0B032A5508CB008B1326
:1003E000831641309B001C141A0883125505031D07
:1003F000DC14831651309B001C141A088312550517
:10040000031DDC108B17CC0B1B2A5608CC008B135A
:10041000831642309B001C141A0883125605031DD4
:100420005C15831652309B001C141A088312560563
:10043000031D5C118B17CD0B332A5708CD008B138E
:10044000831643309B001C141A0883125705031DA2
:10045000DC15831653309B001C141A0883125705B1
:10046000031DDC118B17CE0B4B2A5808CE008B13C3
:10047000831644309B001C141A0883125805031D70
:100480005C16831654309B001C141A0883125805FE
:10049000031D5C128B17CF0B632A5908CF008B13F7
:1004A000831645309B001C141A0883125905031D3E
:1004B000DC16831655309B001C141A08831259054C
:1004C000031DDC128B17D00B7B2A5A08D0008B132C
:1004D000831646309B001C141A0883125A05031D0C
:1004E0005C17831656309B001C141A0883125A0599
:1004F000031D5C138B17D10B932A5B08D1008B1360
:10050000831647309B001C141A0883125B05031DD9
:10051000DC17831657309B001C141A0883125B05E6
:10052000031DDC138B17D20BAB2A5608D2008B139A
:10053000831648309B001C141A0883125505031DAE
:100540005D14831658309B001C141A08831257053B
:10055000031D5D108B17C4015C18C40ADC18C40AA3
:100560005C19C40ADC19C40A5C1AC40ADC1AC40A7D
:100570005C1BC40ADC1BC40A5D18C40AC50146180A
:10058000C50AC618C50A4619C50AC619C50A461AB3
:10059000C50AC61AC50A461BC50AC61BC50A47189E
:1005A000C50A3D1CE92A430845020318E02A45080C
:1005B0004402031808004608DC004708DD00080074
:1005C00043084402031808004608DC004708DD0021
:1005D000080044084502031808004608DC004708E4
:1005E000DD000800C001DE080319DE035E184014B8
:1005F000DE1A40144008C0015E1C4014DE1E401488
:08060000C005C00C5E0C0800EF
:084000000E000300040008009B
:02400E00CC33B1
:10420000FF00FF00FF00FF00FF00FF00FF00FF00B6
:10421000FF00FF00FF00FF00FF00FF00FF00FF00A6
:104220000100FF00FF00FF00FF00FF00FF00FF0094
:10423000FF00FF00FF00FF00FF00FF00FF00FF0086
:104240001000FF00FF00FF00FF00FF00FF00FF0065
:10425000FF00FF00FF00FF00FF00FF00FF00050060
:10426000FF00FF00FF00FF00FF00FF00FF00FF0056
:10427000FF00FF00FF00FF00FF00FF00FF00FF0046
:104280000800800002000800040010000400200064
:1042900004000200FF00FF00FF00FF00FF00FF001E
:1042A00001000100010004000800040010000400E7
:1042B00080000400FF00FF00FF00FF00FF00FF0080
:1042C000FF00FF00FF00FF00FF00FF00FF00FF00F6
:1042D000FF00FF00FF00FF00FF00FF00FF00FF00E6
:1042E000FF00FF00FF00FF00FF00FF00FF00FF00D6
:1042F000FF00FF00FF00FF00FF00FF00FF000000C5
:00000001FF
